:1000000012C02AC029C028C027C026C025C024C0CD
:1000100023C022C021C020C01FC01EC01DC01CC0E4
:100020001BC01AC019C011241FBECFEDCDBF10E0F8
:10003000A0E6B0E0E0EDF2E002C005900D92A0363F
:10004000B107D9F710E0A0E6B0E001C01D92A036DC
:10005000B107E1F7EED03BC1D3CF00C000C000C074
:1000600000C000C000C0000008958C988D9894983E
:10007000959808958C9AF1DF1DD008958D9AEDDF43
:100080008C98EBDF8D98E9DF8C9AE7DF13D0089529
:10009000082E8C9AE2DF802D0DD0882311F002D03B
:1000A000F8CF08958D9A8C9AD8DF8D98D6DF8C98EA
:1000B000D4DF08950894881F01C0880F59F08D9AE5
:1000C00018F400008C9802C08C9A00C0C6DF8D988E
:1000D000C4DFF3CF8D9A8C98C0DF8D98859BFECFBF
:1000E0008827849981E0B9DF99270895882701C07E
:1000F00081E071E08D9A8C98B0DF8D98AEDF8894A6
:1001000084990894771FB0F78D9A813011F08C98FC
:1001100001C08C9AA2DF8D98859BFECF9EDF872F32
:100120009927089591980895919A089584E7A2DFF8
:100130008EE1C0DF80E0BEDFB5DF089584E79ADF9F
:100140008EE1B8DF80E1B6DFADDF089580E0B2DF99
:1001500080E0B0DFA7DF84E78DDF88E0ABDF88E1F8
:10016000A9DFA0DF84E786DF89E0A4DF84EFA2DFD8
:1001700099DF84E77FDF82E19DDF84E09BDF92DF10
:1001800084E778DF85E196DF81E394DF8BDF84E726
:1001900071DF87E18FDF8AE78DDF84DF84E76ADF45
:1001A0008BE188DF8AE086DF7DDF84E763DF8CE137
:1001B00081DF8AE47FDF76DF84E75CDF8EE17ADF50
:1001C00080E078DF6FDF80E090E00895CF93DF93E9
:1001D000EC016817790749F1919820E931E088EC42
:1001E00090E00197F1F721503040C9F7249681E063
:1001F00090E00C2E02C0880F991F0A94E2F7249712
:10020000815F88BB84E736DF88E054DF9E01285E8B
:10021000822F50DF47DF28EE33E088EC90E0019733
:10022000F1F721503040C9F7919ACE01DF91CF917B
:1002300008950F931F93CF93DF9380EF87BB8FE1D8
:1002400088BB899A91988898909A8A98929A8B9A62
:100250008E9A9398969809DF01C024DF84E70ADF1D
:100260008823D9F773DFEC01919A01E010E0809BBD
:1002700008C00130110529F4919860DF00E010E01A
:1002800009C0809907C00115110521F44FDF919A2B
:1002900001E010E0B09905C0BE0180E090E096DF7B
:1002A000EC01B19905C0BE0181E090E08FDFEC0167
:1002B000B29905C0BE0182E090E088DFEC01B399FD
:1002C000D6CFBE0183E090E081DFEC01D0CFFFCF3D
:00000001FF
